** EXPERIMENTAL (HLL) ** Open Watcom Linker Version 1.6beta1 Limited Availability
Portions Copyright (c) 1985-2002 Sybase, Inc. All Rights Reserved.
Created on:       13/11/17 16:25:46
Warning! W1121: file U:/tmp\ldconv__ctypes_obj_1b0c52885a61128c58.obj(U:\DEV\python-2.7.5\Modules\_ctypes\_ctypes.c): '_init_ctypes' has already been exported
Executable Image: build/lib.os2knix-2.7/_ctypes.pyd
creating an OS/2 EMX dynamic link library


                        +------------+
                        |   Groups   |
                        +------------+

Group                           Address              Size
=====                           =======              ====

CGROUP                          0001:00000000        00011670
DGROUP                          0002:00000000        000023b0



                        +--------------+
                        |   Segments   |
                        +--------------+

Segment                Class          Group          Address         Size
=======                =====          =====          =======         ====

TEXT32                 CODE           CGROUP         0001:00000000   00011670
________TEXT           CODE           CGROUP         0001:00011670   00000000
DATA32                 DATA           DGROUP         0002:00000000   000020a0
SET1__os2dll           DATA           DGROUP         0002:000020a0   00000004
SET2__os2dll           DATA           DGROUP         0002:000020a4   00000000
SET3__os2dll           DATA           DGROUP         0002:000020a4   00000004
SET1___CTOR_LIST__     DATA           DGROUP         0002:000020a8   00000004
SET2___CTOR_LIST__     DATA           DGROUP         0002:000020ac   00000000
SET3___CTOR_LIST__     DATA           DGROUP         0002:000020ac   00000004
SET1___DTOR_LIST__     DATA           DGROUP         0002:000020b0   00000004
SET2___DTOR_LIST__     DATA           DGROUP         0002:000020b4   00000000
SET3___DTOR_LIST__     DATA           DGROUP         0002:000020b4   00000004
SET1___crtinit1__      DATA           DGROUP         0002:000020b8   00000004
SET2___crtinit1__      DATA           DGROUP         0002:000020bc   00000000
SET3___crtinit1__      DATA           DGROUP         0002:000020bc   00000004
SET1___crtexit1__      DATA           DGROUP         0002:000020c0   00000004
SET2___crtexit1__      DATA           DGROUP         0002:000020c4   00000000
SET3___crtexit1__      DATA           DGROUP         0002:000020c4   00000004
SET1___eh_frame__      DATA           DGROUP         0002:000020c8   00000004
SET2___eh_frame__      DATA           DGROUP         0002:000020cc   00000014
SET3___eh_frame__      DATA           DGROUP         0002:000020e0   00000004
SET1___eh_init__       DATA           DGROUP         0002:000020e4   00000004
SET2___eh_init__       DATA           DGROUP         0002:000020e8   00000004
SET3___eh_init__       DATA           DGROUP         0002:000020ec   00000004
SET1___eh_term__       DATA           DGROUP         0002:000020f0   00000004
SET2___eh_term__       DATA           DGROUP         0002:000020f4   00000004
SET3___eh_term__       DATA           DGROUP         0002:000020f8   00000004
SET1___fork_parent1__  DATA           DGROUP         0002:000020fc   00000004
SET2___fork_parent1__  DATA           DGROUP         0002:00002100   00000000
SET3___fork_parent1__  DATA           DGROUP         0002:00002100   00000004
SET1___fork_child1__   DATA           DGROUP         0002:00002104   00000004
SET2___fork_child1__   DATA           DGROUP         0002:00002108   00000000
SET3___fork_child1__   DATA           DGROUP         0002:00002108   00000004
________DATA           DATA           DGROUP         0002:00002110   00000000
BSS32                  BSS            DGROUP         0002:00002110   00000280
c_common               BSS            DGROUP         0002:00002390   00000020
________BSS            BSS            DGROUP         0002:000023b0   00000000


                        +----------------+
                        |   Memory Map   |
                        +----------------+

* = unreferenced symbol
+ = symbol only referenced locally

Address        Symbol
=======        ======

Module: U:\usr\lib\dll0hi.obj({standard input})
0001:00000000* __text
0002:00000000* __data
0002:00000000* ___data_start
0002:00002110* ___bss_start
0002:000020a0+ __os2dll
0002:000020a8  ___CTOR_LIST__
0002:000020b0  ___DTOR_LIST__
0002:000020b8* ___crtinit1__
0002:000020c0* ___crtexit1__
0002:000020c8  ___eh_frame__
0002:000020e4  ___eh_init__
0002:000020f0  ___eh_term__
0002:000020fc+ ___fork_parent1__
0002:00002104+ ___fork_child1__
Module: U:/tmp\ldconv__ctypes_obj_1b0c52885a61128c58.obj(U:\DEV\python-2.7.5\Modules\_ctypes\_ctypes.c)
0002:00002390  __ctypes_ptrtype_cache
0002:000023a0  _PyExc_ArgError
0001:0000677b* _PyDict_SetItemProxy
0001:0000681c* _PyDict_GetItemProxy
0001:00006861  __ctypes_alloc_format_string
0001:000068df  _PyCData_FromBaseObj
0001:00007ab7* _PyCData_AtAddress
0001:00007b24  __ctypes_simple_instance
0001:00007b61  _PyCData_get
0001:00007c12  _PyCData_set
0001:00007d21* _PyCArrayType_from_ctype
0001:000080d7  _init_ctypes
0002:00000120* _PyCArray_Type
0002:00000050  _PyCPointer_Type
0002:000001f0* _PyCFuncPtr_Type
0002:000002c0  _PyCData_Type
0002:00000530  _PyCArrayType_Type
0002:00000600* _PyCPointerType_Type
0002:00000390* _PyCFuncPtrType_Type
0002:00000460* _PyCSimpleType_Type
0002:000006d0* _PyCStructType_Type
0002:00002110  __ctypes_conversion_errors
0002:00002114  __ctypes_conversion_encoding
Module: U:/tmp\ldconv_callbacks_obj_1b0c52885a6112d2a8.obj(U:\DEV\python-2.7.5\Modules\_ctypes\callbacks.c)
0001:00008b83  __ctypes_add_traceback
0001:000091f8  __ctypes_alloc_callback
0002:00001330  _PyCThunk_Type
Module: U:/tmp\ldconv_callproc_obj_1b0c52885a6112f1e8.obj(U:\DEV\python-2.7.5\Modules\_ctypes\callproc.c)
0001:0000a7a2  __ctypes_get_errobj
0001:0000a97e  _PyCArgObject_new
0001:0000a9bd  __ctypes_get_ffi_type
0001:0000a9eb  __ctypes_extend_error
0001:0000ab9c  __ctypes_callproc
0002:00001550  _PyCArg_Type
0002:00001400  __ctypes_module_methods
Module: U:/tmp\ldconv_stgdict_obj_1b0c52885a61131128.obj(U:\DEV\python-2.7.5\Modules\_ctypes\stgdict.c)
0001:0000b80e  _PyCStgDict_clone
0001:0000b9fb  _PyType_stgdict
0001:0000ba2a  _PyObject_stgdict
0001:0000bc1b  _PyCStructUnionType_update_stgdict
0002:000018e0  _PyCStgDict_Type
Module: U:/tmp\ldconv_cfield_obj_1b0c52885a611324b0.obj(U:\DEV\python-2.7.5\Modules\_ctypes\cfield.c)
0001:0000e605  __ctypes_get_fielddesc
0001:0000e68d  _PyCField_FromDesc
0002:00001a10* _ffi_type_sint16
0002:00001a50  _PyCField_Type
0002:000019b0  _ffi_type_pointer
0002:000019bc* _ffi_type_longdouble
0002:000019c8* _ffi_type_double
0002:000019d4* _ffi_type_float
0002:000019e0* _ffi_type_sint64
0002:000019ec* _ffi_type_uint64
0002:000019f8  _ffi_type_sint32
0002:00001a04* _ffi_type_uint32
0002:00001a1c* _ffi_type_uint16
0002:00001a28* _ffi_type_sint8
0002:00001a34* _ffi_type_uint8
0002:00001a40  _ffi_type_void
Module: U:\usr\local473\lib\libc_dll.lib(dllinit.obj)
0001:0000eb30  _DLL_InitTerm
Module: U:\usr\lib\libend.lib(src/libend/386/endlink386.asm)
0002:000023b0  _end
0002:00002110  _edata
Module: U:\usr\lib\libend.lib(src/libend/386/end.asm)
0001:00011670* _etext
0001:00011670* __etext
0000:00000000* WEAK$ZERO
0002:000023b0  __end
0002:00002110  __edata
Module: U:\extras\lib\ffi.lib(closures.obj)
0001:0000ed09  _ffi_closure_free
0001:0000f7e2  _ffi_closure_alloc
Module: U:\extras\lib\ffi.lib(prep_cif.obj)
0001:00010b70* _ffi_prep_closure
0001:00010c29  _ffi_prep_cif
Module: U:\extras\lib\ffi.lib(ffi.obj)
0001:00010ce0  _ffi_prep_cif_machdep
0001:00010ddd  _ffi_prep_closure_loc
0001:00010e4a* _ffi_prep_raw_closure_loc
0001:00010e89  _ffi_closure_SYSV_inner
0001:00010f27* _ffi_raw_call
0001:00010fa1  _ffi_call
0001:00011040* _ffi_prep_args
Module: U:\tmp\ldconv_libgcc_a_1b0c52885a6113c0f0.lib(_chkstk_ms.obj)
0001:00011160  ___chkstk_ms
Module: U:\tmp\ldconv_libgcc_so_d_a_1b0c52885a621101d0.lib(emx-ctordtor.obj)
0001:00011190  ___ctordtorInit
0001:000111c4  ___ctordtorTerm
Module: U:\tmp\ldconv_libgcc_so_d_a_1b0c52885a621101d0.lib(emx-eh.obj)
0001:00011200  ___ehInit
0001:00011236* ___ehTerm
Module: U:\extras\lib\ffi.lib(win32.obj)
0001:00011270  _ffi_call_win32
0001:00011350  _ffi_closure_SYSV
0001:00011410  _ffi_closure_raw_SYSV
0001:000114e0  _ffi_closure_STDCALL
Module: U:\tmp\ldconv_libgcc_a_1b0c52885a6113c0f0.lib(_alloca.obj)
0001:00011640  __alloca


                        +----------------------+
                        |   Imported Symbols   |
                        +----------------------+

Symbol                              Module
======                              ======

___libc_ForkRegisterModule          libc065
___init_dll                         libc065
___libc_Back_termDll                libc065
___libc_ForkDeregisterModule        libc065
__atfork_callback                   libc065
_PyExc_TypeError                    python27
_PyErr_SetString                    python27
_PyString_FromStringAndSize         python27
_PyType_Type                        python27
_PyString_FromString                python27
_PyMem_Free                         python27
_PyUnicodeUCS2_FromWideChar         python27
_PySequence_Tuple                   python27
_PyTuple_New                        python27
_PyObject_GetAttrString             python27
_PyErr_Format                       python27
__Py_NoneStruct                     python27
_PyErr_Clear                        python27
_PyCallable_Check                   python27
__PyArg_ParseTuple_SizeT            python27
_PyDict_Update                      python27
_PyObject_IsInstance                python27
_PyType_IsSubtype                   python27
_PyString_AsString                  python27
_PyString_FromFormat                python27
_PyExc_ValueError                   python27
_PyUnicodeUCS2_AsWideChar           python27
_PyUnicodeUCS2_FromEncodedObject    python27
_PyUnicodeUCS2_AsEncodedString      python27
_PyBuffer_Type                      python27
_PyObject_GetBuffer                 python27
_PyBuffer_Release                   python27
_PyDict_DelItem                     python27
_PyErr_WriteUnraisable              python27
__Py_BuildValue_SizeT               python27
_PySequence_SetItem                 python27
_PyObject_CallFunctionObjArgs       python27
_PyDict_GetItemString               python27
_PyDict_Size                        python27
__PyObject_CallMethod_SizeT         python27
_PyInt_FromLong                     python27
_PyObject_CallObject                python27
_PyExc_RuntimeError                 python27
_PyObject_GenericSetAttr            python27
_PySequence_GetItem                 python27
_PyDict_GetItem                     python27
_PyObject_SetAttr                   python27
_PyDict_Next                        python27
_PyMem_Malloc                       python27
_PyObject_SetAttrString             python27
_PyTuple_Pack                       python27
_PyString_Format                    python27
_PyString_InternFromString          python27
_PyErr_NoMemory                     python27
_PyObject_AsReadBuffer              python27
_PyDict_Type                        python27
_PyDict_New                         python27
_PyDict_SetItem                     python27
_PyArg_UnpackTuple                  python27
_PyLong_FromVoidPtr                 python27
_PyDict_SetItemString               python27
_PyLong_AsVoidPtr                   python27
_PyErr_Occurred                     python27
_PyExc_AttributeError               python27
_PyTuple_GetItem                    python27
_PyObject_AsWriteBuffer             python27
_PyObject_IsSubclass                python27
__PyThreadState_Current             python27
__Py_CheckRecursionLimit            python27
__Py_CheckRecursiveCall             python27
_PySequence_Size                    python27
_PyExc_IndexError                   python27
_PyNumber_AsSsize_t                 python27
_PySlice_Type                       python27
_PySlice_GetIndicesEx               python27
_PyString_Concat                    python27
_PyDescr_NewClassMethod             python27
_stpcpy                             libc065
_PyDescr_NewGetSet                  python27
_PyExc_OverflowError                python27
_PyWeakref_NewProxy                 python27
__PyWeakref_ProxyType               python27
__PyWeakref_CallableProxyType       python27
_PyList_New                         python27
_PyUnicodeUCS2_FromUnicode          python27
_PyInt_FromSsize_t                  python27
__PyObject_CallFunction_SizeT       python27
_PyEval_InitThreads                 python27
_Py_InitModule4                     python27
_PyModule_AddObject                 python27
_PyType_Ready                       python27
_PyType_GenericNew                  python27
_PyModule_AddStringConstant         python27
_PyErr_NewException                 python27
_PyObject_GC_UnTrack                python27
_PyObject_GC_Del                    python27
_PySys_GetObject                    python27
_PyFile_WriteString                 python27
_PyErr_Print                        python27
_PyCode_NewEmpty                    python27
_PyThreadState_Get                  python27
_PyFrame_New                        python27
_PyTraceBack_Here                   python27
_PyGILState_Ensure                  python27
_PyExc_RuntimeWarning               python27
_PyErr_WarnEx                       python27
_PyGILState_Release                 python27
__errno                             libc065
__PyObject_GC_NewVar                python27
_PyObject_GC_Track                  python27
_PyArg_ParseTuple                   python27
_Py_BuildValue                      python27
_PyMem_Realloc                      python27
_PyLong_FromSsize_t                 python27
_PyObject_CallMethod                python27
_PyString_Type                      python27
_PyObject_CallFunction              python27
_PyObject_Free                      python27
_PyCapsule_GetPointer               python27
_PyExc_OSError                      python27
___stderrp                          libc065
_PyLong_AsUnsignedLong              python27
_PyLong_AsLong                      python27
__PyObject_New                      python27
_PyThreadState_GetDict              python27
_PyCapsule_IsValid                  python27
_PyCapsule_New                      python27
_PyString_FromFormatV               python27
_PyErr_Fetch                        python27
_PyErr_NormalizeException           python27
_PyObject_Str                       python27
_PyString_ConcatAndDel              python27
_PyErr_SetObject                    python27
_PyEval_SaveThread                  python27
_PyEval_RestoreThread               python27
_PyTuple_Type                       python27
_PySequence_Fast                    python27
_PyObject_GetAttr                   python27
_PyObject_HasAttrString             python27
__PyInt_AsInt                       python27
_PyTuple_Size                       python27
_PyBool_FromLong                    python27
_PyInt_AsUnsignedLongMask           python27
_PyLong_FromUnsignedLongLong        python27
_PyLong_FromLongLong                python27
_PyLong_FromUnsignedLong            python27
__PyFloat_Unpack4                   python27
_PyFloat_FromDouble                 python27
_PyFloat_AsDouble                   python27
__PyFloat_Pack4                     python27
__PyFloat_Unpack8                   python27
__PyFloat_Pack8                     python27
__PyString_Resize                   python27
_PyObject_IsTrue                    python27
_PyFloat_Type                       python27
_PyInt_AsUnsignedLongLongMask       python27
_PyString_Size                      python27
__CRT_init                          libc065
__CRT_term                          libc065
__std_memmove                       libc065
__std_memcpy                        libc065
__std_memcmp                        libc065
__std_wcslen                        libc065
__std_memset                        libc065
__std_sprintf                       libc065
__std_strchr                        libc065
__std_dlsym                         libc065
__std_dlerror                       libc065
__std_strcpy                        libc065
__std_strcat                        libc065
DosRequestMutexSem                  doscalls
DosReleaseMutexSem                  doscalls
DosCreateMutexSem                   doscalls
DosFreeMem                          doscalls
DosQueryMem                         doscalls
DosAllocMem                         doscalls
__std_vsnprintf                     libc065
__std_dlclose                       libc065
__std_fwrite                        libc065
__std_dlopen                        libc065
___ctordtorInit1                    libc065
___ctordtorTerm1                    libc065
__std_abort                         libc065
___register_frame_table             gcc473
___deregister_frame                 gcc473


                        +--------------------+
                        |   Libraries Used   |
                        +--------------------+

U:\extras\lib\ffi.lib
U:\tmp\ldconv_python2_7_dll_a_1b0c52885a61138270.lib
U:\tmp\ldconv_libgcc_a_1b0c52885a6113c0f0.lib
U:\tmp\ldconv_libgcc_so_d_a_1b0c52885a621101d0.lib
U:\usr\lib\libc_alias.lib
U:\usr\local473\lib\libc_dll.lib
U:\usr\lib\libos2.lib
U:\usr\lib\libend.lib


                        +-----------------------+
                        |   Linker Statistics   |
                        +-----------------------+

Stack size:  0000 (0.)
Memory size:  00013a20 (80416.)
Link time: 00:00.12
